:020000040800F2
:1000000078050020810E0008490300084B03000812
:100010004F030008530300085703000800000000C6
:100020000000000000000000000000005B0300086A
:100030005D030008000000005F0300086103000882
:100040009B0E00089B0E00089B0E00089B0E0008EC
:100050009B0E00089B0E00089B0E00089B0E0008DC
:100060009B0E00089B0E00089B0E00089B0E0008CC
:100070009B0E00089B0E00089B0E00089B0E0008BC
:100080009B0E00089B0E00089B0E00089B0E0008AC
:100090009B0E00089B0E00089B0E00089B0E00089C
:1000A0009B0E00089B0E00089B0E00089B0E00088C
:1000B0009B0E0008C10900089B0E00089B0E00085B
:1000C0009B0E00089B0E00089B0E00089B0E00086C
:1000D0009B0E0008F50D00089B0E00083106000875
:1000E0009B0E00089B0E00089B0E0008DFF80CD04A
:1000F00003F02EF900480047D102000878050020DF
:1001000010B501207D490860642000F0D6FD002074
:100110007B49C1F8AC0110BD10B5002479480078C6
:1001200078494978884200DD0124764AD1685068D0
:1001300002F0D2FE00D20124724880687149096938
:10014000884200DD0124204610BD2DE9F04700F073
:100150002BFD0A2190FBF1F06A4908700A21012069
:1001600000F0E6FB8046404602F062FE814602F067
:1001700083FE06464FF06632634B02F0DEFD044616
:1001800002F08DFE5F4948600A21002000F0D0FB9C
:100190008046404602F04CFE814602F06DFE064667
:1001A0004FF06632584B02F0C8FD044602F045FE9F
:1001B00054498860FFF7B0FF10B1FFF7A1FF02E0DC
:1001C00000204E490860BDE8F0872DE9F041002786
:1001D0000026002400254DA14D4802F09CFD4C490D
:1001E000471A4CA14A4802F096FD4949461A00BFF9
:1001F0007C1C07E04648005D303805EB850100EBCC
:100200004105641CB442F5DB2846BDE8F081F0B539
:1002100087B04148008800F40040002844D03FA146
:100220003B4802F078FDD0B13649C86802F024FEA0
:1002300004460D463349486802F01EFE0646314822
:100240000069CDE9044506902E488068CDE900613B
:1002500002902C4842780178324803F0ADF832A180
:100260002B4802F058FD18B1FFF7AFFF2549487041
:100270002FA1274802F04FFD30B1FFF7A6FF04463B
:1002800002F0CDFD1F49C8602BA1214802F043FDBB
:1002900018B1FFF79AFF1B490861C8211C4802F0FA
:1002A0002FFD00201C49088007B0F0BD10B500F0FC
:1002B000C7FC4FF4A06001F079FB4FF4E13000F08F
:1002C0004DFD00F03FF900F054FC00F0D7FA10BDEE
:1002D000FFF7ECFF0120094908604FF47A7000F045
:1002E000ECFC00200649C1F8AC0106E0FFF72DFF49
:1002F000FFF78DFFC82000F0E0FCF7E7AC012142DA
:10030000000021423800002066664A3F28000000B5
:10031000B00000202900000020000020676574491B
:100320006E666F00AC3C000873657454656D7000B8
:10033000736574536D6F6700736574506F69736F85
:100340006E6F757347617300704700BFFEE700BFB3
:10035000FEE700BFFEE700BFFEE77047704770474B
:10036000704700000CB50020019000906C480068B8
:1003700040F480306A49086000BF6948006800F4B2
:10038000003000900198401C0190009818B9019825
:10039000B0F5A06FF1D16248006800F4003010B1F0
:1003A0000120009001E0002000900098012843D136
:1003B0005C48006840F010005A4908600846006830
:1003C00020F0030008600846006840F00200086062
:1003D00053484068524948600846406848600846AB
:1003E000406840F4806048600846406820F47C1013
:1003F00048600846406840F4E810486008460068D5
:1004000040F08070086000BF4548006800F0007050
:100410000028F9D04248406820F003004049486075
:100420000846406840F00200486000BF3C48406811
:1004300000F00C000828F9D10CBD10B5FFF792FFB1
:1004400010BD10B53648006840F00100344908601E
:100450000846406834490840314948600846006809
:10046000324908402E4908600846006820F4802080
:1004700008600846406820F4FE0048604FF41F0002
:100480008860FFF7DAFF4FF000602949086010BD6F
:1004900010B5002100200022214B5B6803F00C0105
:1004A00021B1042906D0082928D107E0214B224C8C
:1004B000236027E01F4B204C236023E0184B5B6830
:1004C00003F47010164B5B6803F48032022303EBD5
:1004D000904022B9194B4343174C23600DE0104B59
:1004E0005B6803F4003323B1144B4343124C236085
:1004F00003E0104B4343104C236003E00D4B0E4CC4
:10050000236000BF00BF064B5B68C3F303130C4CB2
:10051000E15C094B1B68CB40074C236010BD000019
:1005200000100240002002400000FFF8FFFFF6FE2E
:1005300008ED00E000127A000000002000093D00F4
:100540000400002008B501210C2000F0C7FF4FF483
:10055000E040ADF8000010208DF8030003208DF876
:1005600002006946084800F0FDFC4FF40840ADF871
:1005700000006946054800F0F5FC4FF4E0410248F0
:1005800000F09DFD08BD0000000C01400008014086
:1005900010B586B004460121082000F09FFF01211C
:1005A000880400F0A8FF4FF48060ADF81400032029
:1005B0008DF8160018208DF8170005A9874800F05F
:1005C000D1FC4FF40060ADF8140004208DF8170042
:1005D00005A9824800F0C6FC27208DF80000002005
:1005E0008DF8010003208DF8020001208DF8030032
:1005F000684601F0E0F901940020ADF80800ADF87C
:100600000A00ADF80C00ADF810000C20ADF80E009B
:1006100001A9734801F009F8012240F22551704800
:1006200001F09BF801216E4801F08BF806B010BD77
:1006300010B500246A4801F0F5F8C4B269486A4967
:100640000978445468480078401C67490870084697
:100650000078642801DB0020087010BD002004E051
:100660000021604A1154411C88B26428F8DB002143
:100670005D4A1170704710B504460BE000BF402181
:10068000574801F039F90028F9D014F8011B5448F3
:1006900001F0C4F820780028F0D110BD10B5044650
:1006A000FFF7DCFF2046FFF7E6FF50A0FFF7E3FF70
:1006B00010BD10B5044621464A4802F02CFB08B193
:1006C000012010BD0020FCE72DE9F04180460C46DA
:1006D00015461E4600270EE04046FFF7DFFFB0B28A
:1006E00000F0EBFA2046FFF7E4FF10B10120BDE86F
:1006F000F081781CC7B2AF42EEDB0020F7E710B5FF
:10070000642303223AA13BA0FFF7DEFF04464FF427
:10071000167000F0D2FA14B94FF0FF3010BD642308
:10072000032233A135A0FFF7CFFF04464FF4167024
:1007300000F0C3FA14B96FF00100EFE7642303225D
:100740002BA132A0FFF7C0FF04464FF4167000F053
:10075000B4FA14B96FF00200E0E76423032224A185
:1007600032A0FFF7B1FF04464FF4167000F0A5FA6F
:1007700014B96FF00300D1E7642303221CA12FA05A
:10078000FFF7A2FF04464FF4167000F096FA14B972
:100790006FF00400C2E76423032215A12DA0FFF728
:1007A00093FF04464FF4167000F087FA14B96FF007
:1007B0000500B3E70020B1E710B504463223032259
:1007C00028A129A0FFF780FFC82000F076FA204674
:1007D000FFF751FF642000F070FA10BD000C0140DB
:1007E000004800404C000020140000200D000000D4
:1007F0004F4B000041540D0A0000000041542B43B0
:10080000574D4F44453D320D0A00000041542B43E3
:10081000575341503D225A48222C2231323334352D
:1008200036373839222C352C330D0A0041542B43EE
:1008300049504D55583D310D0A00000041542B439D
:1008400049505345525645523D312C353030300DCC
:100850000A00000041542B43495053544F3D300D82
:100860000A0000003E00000041542B43495053450C
:100870004E443D302C31340D0A00000000B587B0E5
:1008800001214FF4027000F029FE4FF4004000F007
:1008900089FD0320ADF8040000208DF8070001A9B0
:1008A0002F4800F05FFB2F4801F0EEF80020029087
:1008B00001208DF80C008DF80D004FF4602004909D
:1008C0000020059001208DF8180002A9254801F0AC
:1008D00002F90121234801F02AF9224801F049F9DF
:1008E00000BF204801F04AF90028FAD11D4801F064
:1008F0004FF900BF1B4801F050F90028FAD107B0AA
:1009000000BD10B50446072301222146154801F019
:100910007AF90121134801F04AF900BF0221114878
:1009200001F0B6FA0028F9D00E4801F0D3F910BD55
:100930002DE9F04107460C460025002608E0384620
:10094000FFF7DFFF0544052000F0B7F9701CC6B2C1
:10095000A642F4DBB5FBF4F080B2BDE8F081000004
:10096000000C0140002401407FB505460C460121E2
:10097000022000F0C0FDADF80850ADF804400020A2
:10098000ADF80A00ADF8060001A9134801F078FBA4
:1009900001221146104801F0EAFE1D208DF80000EA
:1009A00003208DF801008DF8020001208DF803006E
:1009B000684601F000F80121074801F0BDFE7FBD47
:1009C00010B50121044802F080F918B10121024854
:1009D00002F08CF910BD00000004004010B59448EE
:1009E000006820F00F00924908600846006840F057
:1009F0000300086000208F49086040F2EE2000F0FC
:100A000038F901208C49C1F880010F2000F031F93C
:100A100010BD10B500248648006820F00F008449FE
:100A200008600846006840F00800086004E0601CA8
:100A3000C4B2012000F01DF97E488038006808B17A
:100A4000C82CF4DBC82C01DB012010BD002404E01D
:100A5000601CC4B2012000F00CF9764880380068B0
:100A600008B9F02CF4DBF02C01DB0120EDE70020CD
:100A7000EBE710B56E48006820F00F006C49086085
:100A80000846006840F003000860002069490860DB
:100A9000022000F0EEF801206749C1F880016448A7
:100AA000006820F00F00624908600846006840F0C6
:100AB000080008600C2000F0DCF85E488038006810
:100AC00008B1012400E00024322000F0D2F82046D2
:100AD00010BD70B50026012508E0FFF7CAFF0446E7
:100AE000E00140EA6600C6B2681CC5B2082DF4DD1C
:100AF000304670BD70B504464D48006820F00F00C8
:100B00004B4908600846006840F003000860012572
:100B100020E004F0010664106EB100204549086031
:100B2000022000F0A6F801204349C1F880013C20D2
:100B300000F09FF80CE000203E4908603C2000F0E7
:100B400098F801203C49C1F88001022000F091F89A
:100B5000681CC5B2082DDCDD70BD10B5FFF73EFF87
:100B6000FFF757FFCC20FFF7C5FF4420FFF7C2FF78
:100B700010BD08B50121042000F0B0FC0120ADF843
:100B8000000010208DF8030003208DF80200694654
:100B9000274800F0E7F90121254800F090FAFFF717
:100BA0001DFFFFF736FF08BD2DE9F84FFFF7D5FF12
:100BB000FFF714FFFFF72DFFCC20FFF79BFFBE20B0
:100BC000FFF798FFFFF785FF8346FFF782FF044694
:100BD000072C08DDE043C4B26FEA0B0000F0FF0B06
:100BE0004FF0000A01E04FF0010AA1464FEA092048
:100BF0000FFA80F909EB0B000FFA80F9484602F072
:100C00000EF9009002F038F9074600220B4B02F073
:100C100094F8054602F011F90FFA80F9BAF1000FC5
:100C200002D04846BDE8F88FC9F1000000B2F9E7EC
:100C30000008014080012142000021420000E43F01
:100C400010B56FF0040000F000FF2E4800682E4938
:100C5000B0FBF1F02D4908700846007800EB400128
:100C6000C1EBC0104FF6FF7101EAC00028490880AF
:100C700010BD0146254A12784A434FF0E0235A61DD
:100C800000229A611A46126942F001021A6100BFFD
:100C90004FF0E022106900F001021AB100F4803236
:100CA000002AF5D04FF0E022126922F001024FF045
:100CB000E0231A6100229A6170470146144A1288A3
:100CC0004A434FF0E0235A6100229A611A461269A2
:100CD00042F001021A6100BF4FF0E022106900F0FB
:100CE00001021AB100F48032002AF5D04FF0E02260
:100CF000126922F001024FF0E0231A6100229A618A
:100D0000704700000000002000127A00160000204A
:100D100018000020014600BF704700BF544A1288E7
:100D200002F04002002AF9D0C2B2514B1B1D1A80BA
:100D3000704770B505460E46002400BF0BE000BFAB
:100D400040214B4800F0D8FD0028F9D0295D4848E3
:100D500000F064FD641CB442F1DB70BD10B586B0D8
:100D60000446012144F2040000F0B8FB4FF4007087
:100D7000ADF8140003208DF8160018208DF8170028
:100D800005A93C4800F0EEF84FF48060ADF814007F
:100D900004208DF8170005A9364800F0E3F8252057
:100DA0008DF8000003208DF801008DF8020001206D
:100DB0008DF80300684600F0FEFD01940020ADF8B8
:100DC0000800ADF80A00ADF80C00ADF810000C20DA
:100DD000ADF80E0001A9264800F027FC012240F2E0
:100DE0002551234800F0B9FC0121214800F0A9FC5D
:100DF00006B010BD10B540F225511D4800F092FD1F
:100E000010B31B4800F00EFDC4B21B48008800F46C
:100E10000040C8B91848008800F4804060B10A2C2E
:100E200003D000201449088020E01348008840F4D3
:100E300000401149088019E00D2C06D10E480088A9
:100E400040F480400C49088010E00B480088C0F353
:100E50000D000A490C5408480088401C06490880C7
:100E600008460088C72801DD0020088010BD00006A
:100E7000003801400008014020000020B0000020A0
:100E80000648804706480047FEE7FEE7FEE7FEE724
:100E9000FEE7FEE7FEE7FEE7FEE7FEE743040008A5
:100EA000ED00000810B50446CC48844208D1012169
:100EB000042000F02DFB0021042000F029FB46E077
:100EC000C748844208D10121082000F021FB0021FD
:100ED000082000F01DFB3AE0C248844208D10121FD
:100EE000102000F015FB0021102000F011FB2EE077
:100EF000BD48844208D10121202000F009FB0021D7
:100F0000202000F005FB22E0B848844208D10121EE
:100F1000402000F0FDFA0021402000F0F9FA16E030
:100F2000B348844208D10121802000F0F1FA002169
:100F3000802000F0EDFA0AE0AE48844207D101219A
:100F4000801500F0E5FA0021A01500F0E1FA10BDCF
:100F500010B50121084600F0DBFA0021012000F065
:100F6000D7FA10BD2DE9F0410246002500260020E9
:100F700000230024002791F803C00CF00F0591F81E
:100F800003C00CF0100CBCF1000F03D091F802C0AC
:100F90004CEA050591F800C0BCF1000F31D014688F
:100FA00000202BE04FF0010C0CFA00F3B1F800C068
:100FB0000CEA03069E4220D183004FF00F0C0CFA7E
:100FC00003F7BC4305FA03FC4CEA040491F803C0A0
:100FD000BCF1280F06D14FF0010C0CFA00FCC2F84E
:100FE00014C00AE091F803C0BCF1480F05D14FF0DE
:100FF000010C0CFA00FCC2F810C0401C0828D1D328
:101000001460B1F800C0BCF1FF0F34DD546800205B
:101010002EE000F1080C4FF0010808FA0CF3B1F8CB
:1010200000C00CEA03069E4221D183004FF00F0C52
:101030000CFA03F7BC4305FA03FC4CEA040491F8EC
:1010400003C0BCF1280F05D100F1080C08FA0CF818
:10105000C2F8148091F803C0BCF1480F07D100F129
:10106000080C4FF0010808FA0CF8C2F81080401C78
:101070000828CED35460BDE8F0814FF6FF7101809F
:10108000022181700421C1707047024600209368DC
:101090000B400BB1012000E000207047014688683A
:1010A00080B2704702460020D3680B400BB101208C
:1010B00000E0002070470146C86880B270470161B7
:1010C0007047416170470AB1016100E041617047BA
:1010D000C16070474FF480320A438261816182614E
:1010E00082698269704702460020434B18684FF6B8
:1010F0008073184040EA021008433F4B1860704765
:101100003E49C8617047F0B50A460023002400211B
:10111000002500F00046B6F1004F02D1364EF169CD
:1011200001E0354E7168C0F3034583B200F4401608
:10113000B6F5401F08D121F070612F4E766826F079
:1011400070662D4F7E6012E000F48016B6F5801FA9
:1011500006D1032606FA05F4A14341F0706106E0CA
:10116000460D360103FA06F6B14341F0706122B133
:10117000460D360103FA06F6314300F00046B6F19B
:10118000004F02D11C4EF16101E01B4E7160F0BDB9
:1011900030B500228B071C0F0F2303FA04F2164B05
:1011A00008338C1053F824309343134C08348D10BB
:1011B00044F8253023468C1053F824308C07240F34
:1011C00000FA04F423430C4C08348D1044F8253005
:1011D00030BD0A49DC31086070470000000801405A
:1011E000000C0140001001400014014000180140B3
:1011F000001C01400020014000000140000020428E
:10120000DF48006840F00100DD490860084640689A
:10121000DC490840DA49486008460068DA49084075
:10122000D74908600846006820F480200860084616
:10123000406820F4FE0048604FF41F00886070474B
:10124000CF49096821F48031CD4A116011460968FF
:1012500021F480211160B0F5803F03D0B0F5802FDC
:101260000ED106E0C649096841F48031C44A1160D4
:1012700007E0C349096841F4A021C14A116000E0B8
:1012800000BF00BF704710B50146002200230020B8
:101290004A11012A02D1BA4C236806E0022A02D17F
:1012A000B74C236A01E0B64C636A01F01F020124C7
:1012B00094401C400CB1012000E0002010BD38B566
:1012C000002000900024002500BF3120FFF7DBFF45
:1012D00005460098401C00900098B0F5A06F01D022
:1012E000002DF2D03120FFF7CEFF08B1012400E03D
:1012F0000024204638BD01460020A14A106820F095
:10130000F80040EAC10010607047A04908607047CB
:10131000024600209A4B586820F47C1042EA0103F0
:101320001843974B586070479849086670470146C4
:101330000020934A506820F0030008435060704733
:101340008F48406800F00C007047014600208C4A2E
:10135000506820F0F00008435060704701460020BC
:10136000874A506820F4E0600843506070470146A7
:101370000020834A506820F4605040EAC100506069
:10138000704729B17E4A527A02437D4B5A7204E07B
:101390007B4A527A82437A4B5A7270477B49D831E2
:1013A0000860704701460020754A506820F44040AC
:1013B0000843506070470021714A20321170704A12
:1013C00082F82010012802D004280AD104E001216B
:1013D0006B4A2032117005E00521694A20321170F4
:1013E00000E000BF00BF704769490860704764496A
:1013F000096A0143624A11627047654944390860CD
:10140000704730B500210022002400235C4D6D6838
:1014100005F00C0121B1042905D0082923D105E0EC
:101420005C4D056022E05B4D05601FE0544D6D682A
:1014300005F47012524D6D6805F48034022505EBF9
:1014400092421CB9544D554305600BE04C4D6D68FC
:1014500005F400351DB1504D5543056002E04D4D7A
:101460005543056002E04B4D056000BF00BF444D91
:101470006D6805F0F0010909484D6B5C0568DD40B9
:1014800045603F4D6D6805F4E061090A434D6B5CB2
:101490004568DD4085603A4D6D6805F46051C90AC4
:1014A0003E4D6B5C4568DD40C560354D6D6805F4AB
:1014B0004041890B3A4D6B5CC568B5FBF3F505619E
:1014C00030BD29B12E4A526902432D4B5A6104E0C6
:1014D0002B4A526982432A4B5A61704729B1284AE4
:1014E00092690243264B9A6104E0254A926982433D
:1014F000234B9A61704729B1214AD2690243204B9C
:10150000DA6104E01E4AD26982431D4BDA617047FA
:1015100029B11B4AD2680243194BDA6004E0184A29
:10152000D2688243164BDA60704729B1144A1269B7
:101530000243134B1A6104E0114A12698243104BB3
:101540001A61704712494039086070470F49C864F2
:1015500070470B49C87170470948406A40F0807075
:1015600007494862704701460020054A92680A40D0
:101570000AB1012000E000207047014988727047DD
:10158000001002400000FFF8FFFFF6FE000042429C
:101590008004424200127A0000093D00220000202F
:1015A0003200002010B50446FB48844209D10121D5
:1015B0008803FFF7ADFF00214FF48040FFF7A8FF3D
:1015C00032E0F648844209D101214804FFF7ADFF1B
:1015D00000214FF40030FFF7A8FF25E0F0488442D7
:1015E00009D101218804FFF7A0FF00214FF48020DA
:1015F000FFF79BFF18E0EB48844209D10121C804A2
:10160000FFF793FF00214FF40020FFF78EFF0BE060
:10161000E548844208D101210805FFF786FF002133
:101620004FF48010FFF781FF10BD2DE9F04786B021
:1016300005460E460024A24600BFA1460027B089F9
:1016400000B100BF2F462C8A4CF6FF700440F08892
:1016500004432C82AC894EF6F3100440B0883189E3
:101660000843718908430443AC81AC8A4FF6FF40BC
:101670000440B0890443AC8201A8FFF7C2FEC6480B
:10168000874202D1DDF810A001E0DDF80CA0A889A6
:1016900000F4004040B10AEBCA0000EB0A103168C8
:1016A0004900B0FBF1F807E00AEBCA0000EB0A10B2
:1016B00031688900B0FBF1F86420B8FBF0F0040158
:1016C0002009642101FB1089A88900F4004040B181
:1016D000322000EBC900B0FBF1F000F0070004433A
:1016E00008E0322000EB09106421B0FBF1F000F0BB
:1016F0000F0004432C8106B0BDE8F0874FF416516B
:10170000016000218180C18001810C214181002183
:101710008181704710B502460020108A4FF2FF0306
:1017200018400B884C8823438C882343CC88234360
:101730001843108210BD0021018041808180C1804A
:10174000704721B1828942F40052828104E082898B
:101750004DF6FF731A4082817047F0B503460024AE
:1017600000260025002040F66A17B94200D100BFCC
:101770001846C1F3421401F01F06012707FA06F5C7
:10178000012C01D10C3004E0022C01D1103000E01A
:1017900014301AB107682F43076002E00768AF43AF
:1017A0000760F0BD1AB1838A0B43838202E0838A0B
:1017B0008B4383827047028A4FF6F0731A4002828D
:1017C000028A0A430282704782894FF2FF731A40ED
:1017D000828182890A438281704721B1828942F0E5
:1017E0000202828104E082894FF6FD731A408281F1
:1017F0007047028A4FF6DF731A400282028A0A4358
:101800000282704721B1028A42F48042028204E0DF
:10181000028A4BF6FF731A4002827047C1F3080236
:101820008280704701468888C0F30800704781892C
:1018300041F0010181817047028BD2B20283028B99
:1018400042EA012202837047028B02F47F42028344
:10185000028B0A430283704721B1828A42F0200240
:10186000828204E0828A4FF6DF731A4082827047D8
:1018700021B1828A42F01002828204E0828A4FF60D
:10188000EF731A408282704721B1828A42F00802C7
:10189000828204E0828A4FF6F7731A408282704790
:1018A00021B1828942F40042828103E08289C2F33D
:1018B0000E028281704721B1828A42F400628282E4
:1018C00004E0828A4FF2FF731A4082827047828A54
:1018D0004FF6FB731A408282828A0A4382827047E3
:1018E00021B1828A42F00202828204E0828A4FF6AB
:1018F000FD731A408282704702460020B1F5007FD6
:1019000000D100BF13880B400BB1012000E0002084
:10191000704701F40072B2F5007F00D100BFCA43E6
:101920000280704770B50246002400230025002085
:1019300040F66A16B14200D100BFC1F3421501F072
:101940001F03012606FA03F3012D02D196893340C5
:1019500006E0022D02D1168A334001E0968A334018
:101960000C12012606FA04F41688344013B10CB1A7
:10197000012000E0002070BD10B50022002340F6D9
:101980006A14A14200D100BF0A1201249440A3B2FC
:10199000DC43048010BD00000038014000440040DA
:1019A00000480040004C00400050004031490143D5
:1019B000314A1160704770B5002100230F22C478AE
:1019C00004B32D4C246804F4E064C4F5E064210AF7
:1019D000C1F10403CA40447804FA03F18478144046
:1019E00021430901254C0678A155047804F01F0510
:1019F0000124AC4005786D11AD0005F1E025C5F876
:101A0000004109E0047804F01F050124AC401C4D9E
:101A10000678761145F8264070BD1A4A0A400243FE
:101A2000154B1B1F1A60704739B1134A121D1268FB
:101A30000243114B1B1D1A6006E00F4A121D12686B
:101A400082430D4B1B1D1A607047042808D14FF0CC
:101A5000E021096941F004014FF0E022116107E043
:101A60004FF0E021096921F004014FF0E0221161FB
:101A7000704700000000FA050CED00E000E400E013
:101A800080E100E080FFFF1F10B50446FA48844261
:101A900008D101214015FFF73BFD00216015FFF73C
:101AA00037FD17E0F548844208D101210015FFF702
:101AB0002FFD00212015FFF72BFD0BE0F04884429D
:101AC00008D10121C803FFF723FD00214FF4004096
:101AD000FFF71EFD10BD30B5024600200023506800
:101AE000E84C20400D790C6844EA052420435060FE
:101AF0009068E54C2040D1E902542C434D7944EAEA
:101B0000450420439060D06A20F470000C7C641E71
:101B1000E4B2234340EA0350D06230BD00210160AB
:101B2000017141718160C16001210174704721B16F
:101B3000826842F00102826003E0826822F00102C2
:101B40008260704721B1826842F48072826003E053
:101B5000826822F480728260704710B50023CBB295
:101B60001AB144681C43446002E044689C434460EA
:101B700010BD816841F00801816070470146002076
:101B80008A6802F008020AB1012000E000207047D4
:101B9000816841F0040181607047014600208A6835
:101BA00002F004020AB1012000E00020704721B1D8
:101BB000826842F4A002826003E0826822F4A002FC
:101BC00082607047014600208A6802F480020AB1F0
:101BD000012000E00020704710B50A4600210023D4
:101BE000416821F46041531E41EA4331416010BD18
:101BF00021B1426842F40062426003E0426822F48C
:101C0000006242607047F0B504460D460020002196
:101C1000092D11DDE068A5F10A0606EB4607072647
:101C200006FA07F18843A5F10A0606EB460603FA11
:101C300006F10843E0600CE0206905EB4507072644
:101C400006FA07F1884305EB450603FA06F1084357
:101C50002061072A0FDA606B561E06EB86071F26E7
:101C600006FA07F18843561E06EB860605FA06F1CA
:101C70000843606322E00D2A0FDA206BD61F06EBC3
:101C800086071F2606FA07F18843D61F06EB86064D
:101C900005FA06F10843206310E0E06AA2F10D06A0
:101CA00006EB86071F2606FA07F18843A2F10D0608
:101CB00006EB860605FA06F10843E062F0BD21B1A5
:101CC000826842F48012826003E0826822F480120B
:101CD000826070470146C86C80B2704766484C30DD
:101CE0000068704721B1426842F48062426003E0BC
:101CF000426822F480624260704721B1426842F437
:101D00008052426003E0426822F480524260704791
:101D10000A460021816821F4E04111438160704747
:101D200021B1826842F40042826003E0826822F4BA
:101D300000428260704721B1826842F402128260E0
:101D400003E0826822F4021282607047014600209C
:101D50008A6802F400120AB1012000E000207047F6
:101D6000F0B504461546002000220026092911DDA1
:101D7000E068A1F10A0707EB470C072707FA0CF206
:101D80009043A1F10A0707EB470703FA07F2104354
:101D9000E0600CE0206901EB410C072707FA0CF228
:101DA000904301EB410703FA07F210432061A06B57
:101DB000C0F30156EF1C06F1010CA7EB0C0707EB73
:101DC000870C1F2707FA0CF29043EF1C06F1010C59
:101DD000A7EB0C0707EB870701FA07F21043A06394
:101DE000F0BD10B50A4600210023816B21F440119B
:101DF000531E41EA0351816310BD08B500230093CF
:101E00000090009B0B440093009B1A6008BD08B52E
:101E1000024600200090009201F12800009B184427
:101E200000900098006880B208BD0A460021416811
:101E3000164B1940114341607047416282627047FE
:101E40000A460021416821F01F011143416070479B
:101E500040B109490831096841F40001064A0832D5
:101E6000116007E004490831096821F40001024AC1
:101E70000832116070470000002401400028014032
:101E8000003C0140FFFEF0FFFDF7F1FFFFFD3FFFCB
:101E90000246002013680B400BB1012000E0002037
:101EA0007047CA430260704770B5024600200023A5
:101EB00000240B125568CEB205EA060415681D40D1
:101EC00015B10CB1012000E0002070BD00220A1203
:101ED000D34303607047000010B50446FE488442B7
:101EE00008D10121C014FFF713FB0021E014FFF714
:101EF0000FFBC4E0B4F1804F08D101210846FFF781
:101F000014FB00210120FFF710FBB8E0F3488442E6
:101F100008D101210220FFF708FB00210220FFF772
:101F200004FBACE0EE48844208D101210420FFF715
:101F3000FCFA00210420FFF7F8FAA0E0E948844207
:101F400008D101210820FFF7F0FA00210820FFF74F
:101F5000ECFA94E0E448844208D101211020FFF714
:101F6000E4FA00211020FFF7E0FA88E0DF4884421D
:101F700008D101212020FFF7D8FA00212020FFF707
:101F8000D4FA7CE0DA48844208D101214014FFF7FA
:101F9000BFFA00216014FFF7BBFA70E0D548844215
:101FA00009D10121C804FFF7B3FA00214FF4002042
:101FB000FFF7AEFA63E0D048844209D10121080559
:101FC000FFF7A6FA00214FF48010FFF7A1FA56E0C0
:101FD000CA48844209D101214805FFF799FA002136
:101FE0004FF40010FFF794FA49E0C548844208D145
:101FF00001214020FFF799FA00214020FFF795FAD0
:102000003DE0C048844208D101218020FFF78DFACD
:1020100000218020FFF789FA31E0BB48844208D1D3
:1020200001218015FFF781FA0021A015FFF77DFA45
:1020300025E0B648844209D101210804FFF768FA77
:1020400000214FF48030FFF763FA18E0B048844273
:1020500009D101214804FFF75BFA00214FF4003059
:10206000FFF756FA0BE0AB48844208D101218804FF
:10207000FFF74EFA00214FF48020FFF749FA10BD18
:1020800000220288944B98420ED0994B98420BD074
:10209000B0F1804F08D0914B984205D0904B9842B8
:1020A00002D0904B984204D14FF68F731A404B8860
:1020B0001A438D4B984207D08C4B984204D04FF670
:1020C000FF431A40CB881A4302808B8883850B8894
:1020D0000385814B98420BD0854B984208D08B4B9F
:1020E000984205D08A4B984202D08A4B984201D13F
:1020F0000B7A038601238382704770B50024002287
:102100000023058C4FF6FE7635400584028C8388CB
:10211000048B4FF68F752C40B51E2C400D882C4338
:10212000751E2A400D892A434D882A436A4DA842CC
:102130000BD06F4DA84208D0744DA84205D0744D05
:10214000A84202D0734DA84213D14FF6F7752A402A
:102150004D892A434FF6FB752A408D882A434FF656
:10216000FF652B404FF6FF552B408D892B43CD89C2
:102170002B4383800483CD888586028470BD70B52F
:10218000002400220023058C4FF6EF7635400584AD
:10219000028C8388048B48F6FF752C404FF6FF4570
:1021A0002C400D884FF6FF7606EA05252C434FF6A6
:1021B000DF752A400D8906EA05152A434D8806EA8F
:1021C00005152A43444DA84202D0494DA8421DD1CD
:1021D0004FF67F752A404D894FF6FF7606EA0515C2
:1021E0002A434FF6BF752A408D8806EA05152A4313
:1021F0004FF6FF352B404FF2FF752B408D8906EAD5
:1022000085052B43CD8906EA85052B43838004830E
:10221000CD880587028470BD70B50024002200239C
:10222000058C4FF6FF6635400584028C8388848BCD
:102230004FF68F752C404FF6FC752C400D882C43C3
:102240004FF6FF552A400D894FF6FF7606EA052521
:102250002A434D8806EA05252A431F4DA84202D08D
:10226000234DA8421DD14FF2FF752A404D894FF6EC
:10227000FF7606EA05252A434FF6FF352A408D886A
:1022800006EA05252A434EF6FF752B404DF6FF75ED
:102290002B408D8906EA05152B43CD8906EA0515E5
:1022A0002B4383808483CD888587028470BD70B57D
:1022B000002200230024058C4EF6FF76354005846D
:1022C000038C8488828B48F6FF752A404FF6FF45C1
:1022D0002A400D8820E00000002C0140000400404E
:1022E00000080040000C00400010004000140040B6
:1022F00000340140004C01400050014000540140B6
:1023000000180040001C0040002000400040014038
:1023100000440140004801404FF6FF7606EA0525DB
:102320002A434DF6FF752B400D8906EA05352B43F0
:102330004D8806EA05352B43FA4DA84202D0FA4DE6
:10234000A84208D14BF6FF752C408D894FF6FF76D9
:1023500006EA85152C4384808283CD88A0F84050FE
:10236000038470BD828B4FF2FF331A408283828BCD
:102370004FF6FF7303EA01231A4382837047F0B5D7
:102380000C461546002200210026078C4EF6FF7CE5
:1023900007EA0C070784828B018C4FF6FF7707EA68
:1023A000043640F6FF473A404FF6FF7707EA052725
:1023B0003A434FF6FF7707EA03373A43D94FB8421B
:1023C0000ED0D94FB8420BD0B0F1804F08D0D74FC4
:1023D000B84205D0D64FB84202D0D64FB84206D147
:1023E0004DF6FF77394046F48057394305E047F60C
:1023F000FF57394044F48057394382830184F0BD4C
:10240000828B4FF6F3731A408283828B0A43828356
:102410007047F0B50C461546002200210026078CB7
:102420004FF6FF6C07EA0C070784828B018C4FF68E
:10243000FF7707EA04264FF60C773A404FF6FF770E
:1024400007EA03172F433A43B64FB8420ED0B64FB0
:10245000B8420BD0B0F1804F08D0B44FB84205D08D
:10246000B34FB84202D0B34FB84206D14FF6FF5730
:10247000394046F48077394305E04FF2FF57394041
:1024800044F48077394382830184F0BD028B4FF29C
:10249000FF331A400283028B4FF6FF7303EA0123D6
:1024A0001A4302837047F0B50C46154600220021FE
:1024B0000026078C4FF6EF7C07EA0C070784028B97
:1024C000018C4FF6FF7707EA041640F6FF473A40C3
:1024D0004FF6FF7707EA03373A434FF6FF7707EAED
:1024E00005273A438F4FB8420ED08F4FB8420BD0DA
:1024F000B0F1804F08D08D4FB84205D08C4FB84214
:1025000002D08C4FB84206D14FF6DF77394046F003
:102510001007394305E04FF65F77394044F0100764
:10252000394302830184F0BD028B4FF6F3731A40E6
:102530000283028B0A4302837047F0B50C461546AE
:1025400000220021068C4FF6FE773E400684028B67
:10255000018C4FF60C7632407E1C06EA03162E43A1
:102560003243704EB0420ED06F4EB0420BD0B0F13D
:10257000804F08D06D4EB04205D06D4EB04202D0B3
:102580006C4EB04206D14FF6FD76314044F0010664
:10259000314305E04FF6F576314044F00106314312
:1025A00002830184F0BD70B505460C465D48854246
:1025B0000ED05D4885420BD0B5F1804F08D05B4806
:1025C000854205D05A48854202D05A48854200D1FA
:1025D00000E000BF208850B92389A288618828467E
:1025E000FFF7ABFFE1882846FFF79EFF25E0208834
:1025F00004280AD12389A28861882846FFF753FF5F
:10260000E1882846FFF742FF17E0208808280AD112
:102610002389A28861882846FFF7FBFEE1882846C7
:10262000FFF7EEFE09E02389A28861882846FFF7BC
:10263000A6FEE1882846FFF795FE70BD2DE9F04122
:1026400005460C4600260127608808B9022600E0EE
:102650000026A088012801D1022700E00127208858
:10266000A0B92389A28861882846FFF766FFE18820
:102670002846FFF759FF23893A4631462846FFF797
:1026800012FFE1882846FFF701FF13E02389A288A3
:1026900061882846FFF707FFE1882846FFF7F6FE26
:1026A00023893A4631462846FFF747FFE188284606
:1026B000FFF73AFFBDE8F0810A884B881A438B8800
:1026C0001A43CB881A430B891A434B891A438B89C7
:1026D0001A43A0F8442070474FF6FF718180002113
:1026E0000180C180418001727047002101804180DA
:1026F0008180C180018141818181C1817047002138
:1027000001804180012181800021C18001817047C9
:102710000021018041808180C180018141818181CE
:1027200070470000002C01400034014000040040CC
:1027300000080040000C004021B1028842F0010274
:10274000028004E002884FF6FE731A400280704750
:1027500031B1B0F8442042F40042A0F8442005E032
:10276000B0F84420C2F30E02A0F8442070471AB11A
:1027700083890B43838102E083898B438381704784
:102780008182704741EA0203A0F8483070471AB1CD
:1027900083890B43838102E083898B438381704764
:1027A00001894FF6F8721140018170470A460021F5
:1027B00001894FF68F73194011430181704730B57D
:1027C00004460D4629462046FFF7F0FF208940F0D9
:1027D0000700208130BD2DE9F04104460D46164624
:1027E0001F46602D06D13B46012231462046FFF7A9
:1027F0005AFE05E03B46012231462046FFF79DFE8A
:1028000029462046FFF7D2FF208940F007002081AB
:10281000BDE8F08130B50C4600210189C9B24FF600
:10282000FF7505EA0325154325432943018130BD82
:102830002DE9F04105460E461746984600244346CA
:102840003A4631462846FFF7E5FF2C894FF6F870E7
:10285000044044F007044FF68F70044044F07004C5
:102860002C81BDE8F081F0B504460D4616461F46A2
:102870003B46324629462046FFF7CCFF208940F4EC
:1028800080402081F0BD0185828270470A46002188
:1028900001884FF68F731940114301807047F0B5DE
:1028A0000C4615461E460021002200230189028B9A
:1028B000038C4FF6F877394021434FF6FC473A40F6
:1028C00040F201173A434FF6DD773B404FF6FF7772
:1028D00007EA06172F433B43018102830384F0BDBF
:1028E0000A460021018B4FF68F7319401143018373
:1028F00070470A460021018B48F6FF7319404FF6D6
:10290000FF7303EA02231943018370470A4600213B
:10291000818B4FF68F7319401143818370470A46AC
:102920000021818B48F6FF7319404FF6FF7303EACD
:10293000022319438183704721B1028842F080024B
:10294000028004E002884FF67F731A4002807047CD
:1029500021B1828842F00402828004E082884FF62E
:10296000FB731A408280704721B1828842F00802CE
:10297000828004E082884FF6F7731A4082807047A5
:1029800021B1828842F00102828004E082884FF601
:10299000FE731A40828070470A460021018B4FF671
:1029A000F77319401143018370470A460021018BD8
:1029B0004FF2FF7319404FF6FF7303EA02231943E6
:1029C000018370470A460021818B4FF6F773194047
:1029D0001143818370470A460021818B4FF2FF73B8
:1029E00019404FF6FF7303EA0223194381837047AE
:1029F0000A460021018B4FF6FB73194011430183F6
:102A000070470A460021018B4FF6FF3319404FF6FD
:102A1000FF7303EA02231943018370470A4600212A
:102A2000818B4FF6FB7319401143818370470A462F
:102A30000021818B4FF6FF3319404FF6FF7303EAF5
:102A400002231943818370470A460021018B4FF608
:102A50007F7319401143018370470A460021018B9F
:102A6000C1F30E014FF6FF7303EA022319430183FA
:102A700070470A460021818B4FF67F73194011433E
:102A8000818370470A460021818BC1F30E014FF606
:102A9000FF7303EA02231943818370470A4600212A
:102AA000018C4FF6FD7319401143018470470A46AB
:102AB0000021018C4FF6F7731940114301847047D0
:102AC0000A460021018C4FF6DF7319404FF6FF7361
:102AD00003EA02131943018470470A460021018C5E
:102AE0004FF67F7319404FF6FF7303EA0213194341
:102AF000018470470A460021018C4FF6FF531940AC
:102B00004FF6FF7303EA02231943018470470A4614
:102B10000021018C4FF2FF7319404FF6FF7303EA57
:102B200002231943018470470A460021018C4DF6A7
:102B3000FF7319404FF6FF7303EA02331943018410
:102B4000704730B5002301248C40A3B2048C9C4311
:102B50000484048C02FA01F5ADB22C43048430BD28
:102B600030B5002304248C40A3B2048C9C4304841D
:102B7000048C02FA01F5ADB22C43048430BD70B56B
:102B80000346002000241846183001258D40ACB2C1
:102B90001D8CA5431D8409B1082909D100EB6100F2
:102BA000056825F0700505600568154305600EE0B1
:102BB0000D1FC5F34E052844056825F4E045056062
:102BC00005684FF6FF7606EA02263543056070BDBC
:102BD00021B1028842F00202028004E002884FF62E
:102BE000FD731A400280704721B1028842F004024E
:102BF000028004E002884FF6FB731A40028070479F
:102C000021B1828842F08002828004E082884FF6FF
:102C10007F731A408280704702884FF6F7731A401C
:102C2000028002880A430280704782884FF68F73C1
:102C30001A40828082880A438280704702894FF658
:102C4000F8731A40028102890A430281704702899F
:102C50004FF67F731A40028102890A43028170474E
:102C600081847047818570478186704701877047EE
:102C700081877047A0F84010704702884FF6FF43E5
:102C80001A40028002880A43028070470146888EFB
:102C900070470146088F70470146888F704701468C
:102CA000B1F8400070470146888C70470146088D96
:102CB000704702460020138A0B400BB1012000E050
:102CC00000207047CA430282704730B50246002098
:102CD00000230024158A05EA0103958905EA010409
:102CE00013B10CB1012000E0002030BDCA430282C4
:102CF0007047D2B201E000F8012B491EFBD27047A9
:102D00000022F6E710B513460A4604461946FFF7B7
:102D1000F0FF204610BD30B505462A460B4612F896
:102D2000010B13F8014B08B1A042F8D01CB10028E8
:102D300002D06D1CF1E7284630BD2DE9FE4F81EA37
:102D4000030404F0004421F0004100944FF0000B14
:102D500023F0004350EA01045ED052EA03045BD042
:102D6000C3F30A54C1F30A552C44A4F2F33401947A
:102D7000A0FB0254C1F3130141F48011C3F3130308
:102D800043F4801301FB024400FB034E840A970ABC
:102D900044EA815447EA8357A4FB076802958D0AE9
:102DA00005FB07854FEA932C04FB0C542705029D75
:102DB0004FEA065847EA1637B5EB08056EEB070CE5
:102DC000870E920E47EA811742EA8312A7FB02019F
:102DD000B6EB0B0164EB00042B0D43EA0C335E18D9
:102DE00044EB1C50DA465146E7FB0201C5F31304DD
:102DF0004FEA0B3343EA14534FEA0432019C43EA8F
:102E00000603A4F10C040294009CCDE900B400F088
:102E10000AF903B0BDE8F08F00200146F9E7C10FC1
:102E200080EAE0700844CA079623002100F0BEB88B
:102E300096230022114600F0B9B870B5C1F30A52CA
:102E400001F000450024C1F3130140F2FF3341F4C7
:102E500080119A4201DA002070BD40F233439A4259
:102E6000A2F2334203DC524200F087F800E09040C7
:102E70002C43F1D0404270BD00F0004230F00040E1
:102E80000AD0C10D01F56071C0F3160042EA01518C
:102E9000C20840071143704700200146704701F007
:102EA000004330B421F0004150EA010206D00A0D7F
:102EB000A2F56072C1F31301002A02DC30BC0020CD
:102EC0007047440F44EAC104C100E01830BC00EB75
:102ED000C25000F062B80000002801DBC0F10040E1
:102EE000002901DBC1F100418842704730B50B4633
:102EF000014600202022012409E021FA02F59D422A
:102F000005D303FA02F5491B04FA02F52844151EFD
:102F1000A2F10102F1DC30BD2DE9F05F0546002091
:102F200092469B4688460646814640241BE028463A
:102F300041464746224600F020F853465A46C01AFA
:102F4000914110D311461846224600F013FA2D1A6B
:102F500067EB01084F4622460120002100F00AFAE3
:102F600017EB00094E41201EA4F10104DFDC4846A6
:102F700031462A464346BDE8F09F202A04DB203A2A
:102F800021FA02F00021704721FA02F3D040C2F189
:102F9000200291400843194670470029A8BF704796
:102FA000401C490008BF20F00100704710B4B0FA7F
:102FB00080FC00FA0CF050EA010404BF10BC70471A
:102FC00049B1CCF1200421FA04F411FA0CF118BF34
:102FD000012121430843A3EB0C01CB1D4FEA006103
:102FE0004FEA102042BF002010BC704700EBC350D6
:102FF00010440029A4BF10BC7047401C490008BF02
:1030000020F0010010BC704710B5141E73F10004CD
:1030100008DA401C41F1000192185B411A4301D1CA
:1030200020F0010010BD2DE9F04D92469B4611B1F4
:10303000B1FA81F202E0B0FA80F22032904600F05C
:1030400099F904460F4640EA0A0041EA0B0153464B
:103050005A46084313D0114653EA010019D0C8F16B
:1030600040025046FFF789FF05460E465046594636
:10307000424600F07FF9084305D0012004E02046D5
:103080003946BDE8F08D0020054346EAE0762C4342
:1030900037430A986305E40AA0EB08000022FD0A02
:1030A00044EA47540A3002D500200146E9E7010509
:1030B00010196941DDE9084500196941BDE8F04D85
:1030C000A2E72DE9FE4F804681EA0300C00F0C46BF
:1030D000009021F0004123F00045B8EB0200A94127
:1030E00005D24046214690461C460B46024623F038
:1030F0000040104347D0270DC7F30A00C3F30A511D
:103100000290401A019040286BDAC3F3130040F498
:10311000801B0098924620B10023D2EB030A63EB98
:103120000B0B01985946C0F14002504600F022F9BD
:1031300006460D4650465946019A00F02AF910EB12
:1031400008006141002487EA115284EAE7731A43B8
:1031500040D0009A62B3019A012A4FEA075215DC67
:10316000001B61EB02014FF0004202EA0752CDE979
:103170000042001C41F5801132462B46FFF753FFF9
:1031800003B0BDE8F08F40462146F9E7001B61EB34
:103190000201001C41F5801300185B412018A2F5C4
:1031A000001747EB030140EAD570B6196D4111E0F5
:1031B0006D084FEA360645EAC0754FEA0752001B14
:1031C00061EB0201001C41F5801149084FEA300013
:1031D0000019514132462B4603B0BDE8F04FFFF7CE
:1031E00013BF0098012240000023D0EB020263EBE2
:1031F000E073009821464FEAE074B8EB000061EB01
:103200000401E9E783F000435BE781F0004158E700
:103210002DE9F04D81EA030404F0004B21F0004554
:1032200014464FF0000A23F0004150EA050220D076
:1032300054EA01021DD0C5F30A570246C5F3130331
:10324000C1F31300C1F30A5640F4801543F4801310
:10325000A7EB0608101BD64608F2FD3873EB0500F5
:1032600002D308F1010801E092185B41B8F1000FA8
:1032700003DA00200146BDE8F08D00204FF48011F4
:10328000064684460EE0171B73EB050705D3121B99
:1032900063EB050306434CEA010C49084FEA300092
:1032A00092185B4150EA0107EDD152EA030012D0B7
:1032B00082EA040083EA0501084305D0101BAB41F4
:1032C00006D20122002306E000224FF0004302E074
:1032D0006FF0010253101AEB06004CEB085110EB93
:1032E0000A0041EB0B01BDE8F04DFFF78DBEC1F3C5
:1032F0000A52C1F3130140F2FF3341F480119A42A4
:1033000002DA00200146704740F233439A42A2F2AB
:10331000334202DC5242FFF730BE00F02BB800000F
:1033200030B5041E71F1000404DB4FF0004440424C
:1033300064EB0101141E73F1000405DB1C464FF021
:103340000043524263EB0403994208BF904230BDF0
:10335000064C074D06E0E06840F0010394E80700E2
:1033600098471034AC42F6D3FCF7C4FE143D000875
:10337000343D0008202A04DB203A00FA02F1002044
:1033800070479140C2F1200320FA03F319439040A3
:103390007047202A06DBCB17203A41FA02F043EAB5
:1033A000E07306E041FA02F3D040C2F120029140FE
:1033B00008431946704700000FB4054B10B503A928
:1033C000044A029800F0DAF810BC5DF814FB000023
:1033D0001B0D00081C00002002E008C8121F08C1D5
:1033E000002AFAD170477047002001E001C1121F86
:1033F000002AFBD1704700002DE9FF5F82B0002159
:10340000DDE90430020DDDF840B0034318D044F686
:103410001050A2F2FF3242431514119801281FD018
:10342000A5EB0B00401C5FEA000A4FF000064E4F70
:10343000DFF83891B046504615D5CAF1000413E0C4
:10344000119801244AA3012801D16FEA0B010298C7
:10345000119AC0E90031C0E9024206B0BDE8F09F10
:10346000CBF10000DFE704460021404A491842EB57
:103470000450CDE9001012E0E00707D032463B4689
:1034800040464946FFF759FC8046894632463B464E
:1034900010461946FFF751FC06460F466410002CF3
:1034A000EAD1DDE90401DDE90023BAF1000F06DA13
:1034B000FFF743FC42464B46FFF73FFC05E0FFF7B2
:1034C000A7FE42464B46FFF7A3FE04460E460022E7
:1034D000284BFFF725FF03D84FF0FF30014607E0E8
:1034E0000022254B20463146FFF7EBFDFFF7FFFE9C
:1034F000102409E0002C0ADB0A220023FFF70CFD50
:10350000039B30321A55641E50EA0102F2D1641C4A
:10351000039AC4F111031444119A012A03D0012221
:1035200008430DD10AE0084304D000204FF0110BEE
:10353000119072E7A3EB0B056D1E0DE05B4504DDFA
:103540004FF0000205F1010504E003DA4FF000023C
:10355000A5F10105002AECD002981199C0E90231C9
:10356000C0E9004579E70000000014400000F03F8A
:10357000300000000000F0430000E03F2DE9FF4F65
:1035800095B09B468946064600250FE2252877D14F
:1035900000242746F84A0121059400E0044316F868
:1035A000013F203B01FA03F01042F7D130782A287E
:1035B00011D06FF02F033078A0F13002092A16D80D
:1035C000059A44F0020402EB820203EB420210442B
:1035D000761C0590EFE759F8042B0592002A03DAD0
:1035E000504244F40054059044F00204761C3078B4
:1035F0002E2816D116F8010F44F004042A280DD005
:103600006FF02F023078A0F13003092B09D807EBB7
:10361000870302EB4303C718761CF3E759F8047BD2
:10362000761C30786C280FD006DC4C2817D0682820
:103630000DD06A2814D104E0742810D07A280FD154
:103640000DE044F400140AE044F4801401E044F472
:1036500040147278824202D104F58014761C761CE4
:10366000307866280BD013DC582877D009DC002886
:1036700075D04528F6D04628F4D047281AD19DE1C8
:1036800018E0632835D0642879D0652812D195E1F7
:10369000702873D008DC6728F1D069286FD06E28B5
:1036A0000DD06F2806D1B5E073282CD0752875D0C1
:1036B000782874D05A46179990476D1C75E1C4F369
:1036C0000250022809D003280DD0D9F80010042890
:1036D0000DD00D6009F1040967E1D9F80010EA176F
:1036E000C1E90052F6E7D9F800100D80F2E70D703D
:1036F000F0E719F8041B8DF8001000208DF8010088
:10370000EA46012003E059F804AB4FF0FF306107AF
:103710004FF0000102D40DE008F101018846B942E2
:103720000FDA8045F8DB1AF808100029F4D108E018
:1037300008F1010188468142FADB1AF808100029D5
:10374000F6D105985B46A0EB080721463846179A44
:1037500000F094FA284400EB080507E04DE029E169
:103760000DE01AF8010B5A4617999047B8F1010875
:10377000F7D25B4621463846179A13E142E00A2207
:103780000092C4F302524FF0000A022A08D059F8FE
:1037900004CB032A4FEAEC710AD00DE029E02AE0BD
:1037A00009F1070121F00702F2E802C1914609E0A0
:1037B0000FFA8CFC4FEAEC71042A03D14FFA8CFC0F
:1037C0004FEAEC71002907DA0A460021DCF1000C0F
:1037D00061EB02012D2202E0220504D52B228DF897
:1037E0000420012203E0E20701D02022F7E79046FF
:1037F00059E00A2102E010220DE010214FF0000AEA
:1038000000910BE010224FF0000A44F00404082756
:10381000009203E008224FF0000A0092C4F3025223
:10382000022A05D059F804CB0021032A08D009E068
:1038300009F1070121F00702F2E802C1914605E013
:103840001FFA8CFC042A01D10CF0FF0C4FF0000889
:10385000220728D5702806D0009B83F0100353EA76
:103860000A0305D00EE040228DF80420012208E072
:103870005CEA010206D030228DF804208DF80500A4
:1038800002229046009B83F0080353EA0A030AD100
:103890005CEA010201D1620705D530228DF80420CF
:1038A0004FF001087F1E582804D034A003900EA8C2
:1038B00002900DE036A0F9E753466046009AFFF704
:1038C0002BFB84460398825C0298401E0290027093
:1038D0005CEA0100F0D1029806A9081A00F1200A5A
:1038E000600702D524F4803400E00127574502DD4B
:1038F000A7EB0A0000E0002000EB0A010090059809
:103900004144401A0590E00306D45B462146179ACD
:10391000059800F0B3F90544002706E001A85A46CF
:10392000C05D179990476D1C7F1C4745F6DBE0038F
:103930000CD55B462146179A059800F09FF905447F
:1039400004E030205A46179990476D1C0099481E94
:1039500000900029F5DC08E0029802995A460078A8
:10396000491C0291179990476D1CBAF10001AAF108
:10397000010AF1DC65E10000092801003031323331
:10398000343536373839616263646566000000009B
:103990003031323334353637383941424344454685
:1039A0000000000000F058F90544761C307800282B
:1039B0007FF4ECAD19B02846BDE8F08F620700D463
:1039C000062709F1070222F0070CFCE80223E14672
:1039D00003F000485FEA080C02D00FF2702C0DE0F3
:1039E0005FEA045C02D50FF2682C07E05FEAC47C52
:1039F00002D00FF2602C01E0AFF2700C4FF0FF38F4
:103A000023F00043CDF850C065280CD006DC4528D3
:103A100009D046281DD047283DD13DE0662818D062
:103A200067287ED138E00021112F01DB112000E052
:103A3000781CCDE9000106A90EA8FFF7DDFCDDE941
:103A40000F010E9A03910021009207F1010A0491DF
:103A50004DE04FF000400097CDE9011006A90EA8F7
:103A6000FFF7CAFCDDE90F0203920E9B11990022B9
:103A7000DDF80CA00093049211B9791C00EB010A47
:103A8000B7EB0A0004D4C0F1FF3007F1010A04903B
:103A9000AAEB0700019044E0012F00DA0127002182
:103AA000112F01DD112000E03846CDE9000106A903
:103AB0000EA8FFF7A1FCDDE90F010E9A039100218A
:103AC00004910092BA4621070CD40399514500DABB
:103AD0008A46BAF1010F05DD009AAAF10101515C95
:103AE000302908D0B84202DA10F1040F06DA0121B9
:103AF000CDE9011015E0AAF10101E9E7002805DC94
:103B0000049901440491AAEB000102E0411C5145D3
:103B100000DD8A460499401A401C01904FF0004095
:103B20000290200704D40198504501DBCDF80480B1
:103B300000208DF84F0002980DF14F07B0F1004FB3
:103B400025D02B200E9002984FF0020800280CDAA6
:103B5000404202902D200E9007E00A210298FFF7C4
:103B6000C5F93031029007F8011DB8F10001A8F144
:103B70000108F2DC02980028EFD1791E0E98087037
:103B8000307800F0200040F0450007F8020D12A840
:103B9000C01B00F107081498007800B1012000EB69
:103BA0000A01019801EBE07105984144401A401E5A
:103BB0000590E00306D45B462146179A059800F06D
:103BC0005DF805441498007818B15A461799904743
:103BD0006D1CE00324D55B462146179A059800F03A
:103BE0004DF805441CE00498002807DBDDE90301DB
:103BF000884203DD0098405C179901E01799302056
:103C00005A469047049805F10105401C049001981C
:103C1000401E019004D12E205A46179990476D1CE2
:103C2000BAF10001AAF1010ADDDC05E017F8010B89
:103C30005A46179990476D1CB8F10001A8F1010888
:103C4000F4DC5B462146179A0598ABE62D00000090
:103C50002B000000200000002DE9F0410446002563
:103C60001E461746880404D405E039462020B04794
:103C70006D1C641EF9D52846BDE8F0812DE9F041A0
:103C8000044600251E469046C80301D5302700E0B3
:103C90002027880404D505E041463846B0476D1C0E
:103CA000641EF9D52846BDE8F081000074656D708A
:103CB0003A25642C2074656D705F74687265736852
:103CC0006F6C643A25642C736D6F673A25302E3221
:103CD000662C20506F69736F6E6F75734761732523
:103CE000302E32662C20736D6F675F746872657357
:103CF000686F6C643A25642C20506F69736F6E6F27
:103D000075734761735F7468726573686F6C643A4A
:103D100025640000343D0008000000203800000049
:103D2000D83300086C3D0008380000204005000032
:103D3000E833000800A24A04000000000000000070
:103D4000010203040607080900000000000000004B
:103D50000000000000000000000001020304010256
:0C3D60000304060708090204060800001E
:04000005080000ED02
:00000001FF
